:06000000022FFD02033C8B
:03000B0002008070
:0300130002034F96
:03001B000200B030
:03002B0002030AC3
:03005B0002035E3F
:030073000203295C
:20008000C0D075D01018B8CF0408208507B285868AD0D03253A4DFD285C2A98F8E7589AAAE
:2000A000C289C28B758A00D2A8D2AAC228D0D032C2A8C28E85578BC0D075D008C0E0C0F0A9
:2000C000C2CAA9CEAACFD2CAC3E99558F9EA95597049C3E9955A4043955A503FB8103C78CD
:2000E00000A9567D00E2FEC39DC399402E99EC33FC08E2FDC39EC399402199EC33FC08E223
:20010000FEC39DC399401499EC33FC08E2FDC39EC399400799EC33FC088002806AE2FEC367
:200120009DC399406299EB33FB08E2FDC39EC399405599EB33FB08E2FEC39DC399404899C2
:20014000EB33FB08E2FDC39EC399403B99EB33FB08E2FEC39DC399402E99EB33FB08E2FD0A
:20016000C39EC399402199EB33FB08E2FEC39DC399401499EB33FB08E2FDC39EC39940071A
:2001800099EB33FB08801E0530E53070021530C3E5309432400AD225755B00755C0041FA4B
:2001A00075310A41FAE2FEC39DC39940DA99EA33FA08E2FDC39EC39940CD99EA33FA08E2A3
:2001C000FEC39DC39940C099EA33FA08E2FDC39EC39940B399EA33FA08EBC46B6C6A30271F
:2001E00001F4540F70A1C3EBF4FA9460FBECF4540F9400FC5018EA7C007B00600CC313505D
:2002000007B55B05055C8006E4F55B755C0030221BC3EB94D0F5F0EC94074003ABF0FC30E1
:200220002101B39226C3EB33FBEC33FCEB54F04CC475F00584FAEC13FCEB132AFBEC3400D5
:20024000FC30E3047BFF7C07201C27301124EC700C798187F0C3EB95F05002ABF0E5376051
:200260001175F028A42BFBEC3400FC30E3047BFF7C07EB54F84CC423F97007EB7004D225B6
:200280008005753200C225E53060021530C3E54CFD954D4002AD4DC3ED995002EDF9E9F422
:2002A000F97A00302914EBF4540724C0F8E623F630E007E92401F9700119C3E99405FBEA77
:2002C0009400FC5005E4FBFC800DC3EB954FEC95504004AB4FAC5089FC8BEA75310A302733
:2002E00019302816758E017589A2D28543A420780085638AC28DD2A980097800758A00D2EF
:20030000A8D2AAD0F0D0E0D0D032C0E0C2CF053BD223E5317004D22580021531302507E587
:20032000320460020532D0E032C2AF53E67F53917F7592FA7593FFC218D2AF32C0E0E58ADC
:2003400085578BC0D075D008F208D0D0D0E032C2AAD28EC2CA85CE5885CF59D2CA32327AB3
:20036000007901801E7A00790580187A00790A80127A007964800C7A0079C880067A00792F
:20038000FA8000090A8009781874FFD5E0FDD8F9D9F5DAF3227A427B3580247A2D7B4D8005
:2003A0001E7A267B5C80187A197B8C80127A147BAF800C7A427B1E80067A2D7B2C8000E512
:2003C000537001227902E4D293D5E0FDD292D5E0FDC292D5E0FDC293D5E0FDE920E002D2E1
:2003E0009030E002D294E553D5E0FDE920E002C29030E002C2947496D5E0FDD9C9EA78C8DE
:20040000D8FED5E0F9DBBDD293227195719B71A12271B971952271A1719B719522799987C2
:2004200053B8010471958017B80204719B8010B8030471A18009B8040471A7800271AD796A
:2004400098875322903070E493F4601D7C3E903074E493A3FB6012E493FA600471BF8006F0
:20046000EBF97A007183A3DCE82278A5E6F954037000E9540C7000E954307000E954C070DB
:200480000022C290C292C294D291D293D29575D5FF22201E2E78FF201026E53A6022E542A3
:2004A000601E74FF301102747F8542F084853AF0A4F8C5F0600278FFC3E8954E5002A84E2B
:2004C000884D22C3E54194A0E5429400E54D5003148001046002F54D22102301220566E5C3
:2004E000665403B4012CE551604F7552FFE5BE6048E5BDC3955140417552C89404403A7586
:200500005296940440337552649404402C7552328027B4021EE5516020C3E54C955260193B
:200520004008E54C6013154C800FE54C046002054C8006B4030375E895302438E566541F7B
:20054000B40412E5BE7003E48004E5BD9414F564756502801FB4080875648875650880149A
:20056000B40C087564AA75650A8009B410067564CC75650C227541007542F022C2AFC2CAD0
:20058000A8CEA9CFAA3B30CF010AD2CAD2AFC3EA13FAE913F9E813F8201014C3E8953C8877
:2005A0003CF8E9953D893D547FF9301E36C196AB3CAC3DAD3E883C893D8A3EC3E89BE99C07
:2005C000EA9D547F60087541FF7542FFC165AE3FAF408B3F8C40C3E89EF8E99FF9AA41ABFE
:2005E000428011AA41AB42C3EB9404404894044013201126C3EB13FDEA13FCC3ED13FDECDD
:2006000013FC804AEBC423FCEAC423541F4CFC7D00C3E913F9E813F88034EBC423FC541F8A
:20062000FDEC54E0FCEAC423541F4CFCC3E913F9E813F88019EBC4FCEAC4540F4CFC7D0050
:20064000C3E913F9E813F8C3E913F9E813F8C3EA9CFAEB9DFBEA28F541EB39F54250067510
:2006600041FF7542FFC3E54294025002D21EE542C4FA540FFBEA54F0FAE541C4540F4AFAC6
:20068000C3EA9402FAEB9400FB40057048EA70457A017B00803FAA41AB42EBC4FCEAC454CD
:2006A0000F4CFCC3EA9CFAEB9400FBE80303543F2AFAEB3400FB8A418B42C394024002C272
:2006C0001EEBC4FE7B00EAC4540F4EC39402FA400270027A01202806301808120AA0301851
:2006E0000280FB854892854993D21843E6807892E6FFC3E49AF8E49BF9C3E833F8E933F99F
:20070000201E7F3010047F038015C3E5389482400E0F941E40010FC3EF940640027F05E872
:20072000FAE9FBD3E913FDE813FC8C468D4788488949C3EF9403602BEF20E00CE82CF8E90C
:200740003DF9ECFAEDFB800BE8D338F8E939F97AFF7BFFC3EF9403400A8A4A8B4B8844897F
:20076000458050884A894B8A448B45301045754AF0754BFF7546F07547FF7548F07549FF5D
:200780008031E8FAD313FC8C468848C3EF9403601EEF20E007E82CF8ECFA8007E8282401D7
:2007A000F87AFFC3EF940340068A4A88448004884A8A44202806301808120AA03018028051
:2007C000FB753502D21843E68030112DA841A942C3E913F9E813F8301004E92440F9C2AFF7
:2007E00053E67F759100C3E498F594E499F595759104D21843E680D2AF2275F000301D0E6C
:2008000075F040800975F040301D0375F000D2197543007A027B02201E1D301102C219300B
:2008200010067A367B36800F7B28E542700104FAC3942840027A28201811E543600D3010F8
:2008400003D53504D21A80671207C40543E59B5440B5F00DE53460BB2019B8DADAC21A8094
:200860004E20100B2019110AC3EA9B40CA80A40AC3EA9B40011A80BFC21953E67F759100A0
:20088000301E117594007595F0759104D21843E680020813E5427EFFC3334009C33340051E
:2008A000C3334001FEC3E49E759400F59580DAC2AF53E67F854492854593759100854A9487
:2008C000854B95759104D21843E680D2AF201013301A1220110F201D0C20190915811581FF
:2008E0000211EF053422E53875F007A430190105F0A2F013A2F113A2F213F538C3947850F1
:2009000003753878C3E53895394009C290C292C29475D5FF20280530180751A0301802801C
:20092000FB854692854793D21843E6802220120FC2AFD293C29175D5CFD2AF759F1022C23F
:20094000AFD293C29575D5FCD2AF759F102220120FC2AFC29475D5F3C291D2AF759F1122BF
:20096000C2AFC29075D5F3C295D2AF759F122220120FC2AFD291C29575D5F3D2AF759F1207
:2009800022C2AFD295C29175D5F3D2AF759F112220120FC2AFC29275D5FCC295D2AF759FCD
:2009A0001022C2AFC29275D5CFC291D2AF759F102220120FC2AFD295C29375D5FCD2AF7563
:2009C0009F1122C2AFD291C29375D5CFD2AF759F122220120FC2AFC29075D5CFC293D2AF47
:2009E000759F1222C2AFC29475D5FCC293D2AF759F11227432A28540032085F750033085D1
:200A0000F2D5E0F3922722E55B700122F8C39406500FC2AF12048212041D120377D2AF8011
:200A200078C3E55C94064077B80704C221806AB80804D2218063B80904C222805CB80A0474
:200A4000D2228055B80D0A75640075650ED2248048B80E0A7564FF75650EC224803BB81482
:200A60000A7988E714A2E09221802EB8150B7988E714A2E0B392218020B80C1DE4A2219217
:200A8000E0A22292E1047988F77554A57555F1B109755400755500D2AF755B00755C002289
:200AA000C0D075D010BE002DE5657022C2AF854126854227D2AFE526A23813F9A2391329B6
:200AC000F526E52703C2E7F903C2E739F5270E201803D0D022BE0124E5657010E527705DB8
:200AE000E526701175270F7526FF80098564268565277565000E201803D0D022BE0215E5DD
:200B000026C465266527F478D0A65D71BA0E201803D0D022BE030BE52671BA0E201803D044
:200B2000D022BE040CE526C471BA0E201803D0D022E52771BA087E00D0D0D2282220E7165A
:200B400020E61D20E52720E43420E34120E25020E15CE52641F5A23733F52675270F41F5D2
:200B6000A23733A23633F52675270D41F5A23733A23633A23533F52675270B41F5E52654EC
:200B8000F0C23C4527C4F52675270941F5E526A23813A23913A23A13F52675270741F5E593
:200BA00026A23813A23913F52675270541F5E526A23813F52675270341F5540F23900BC178
:200BC0007361E161EB61F8810981138120812A813E814B815F816681778181819881A28148
:200BE000B608A65F08A65D08A65D2208A65D08A65E08A65D08A65D2286F0E55EB5F002E566
:200C00005FF608A65F08A65D2208A65D08A65F08A65D2208A65E08A65D08A65D08A65D22B1
:200C200008A65E08A65E08A65D2286F0E55EB5F002E55FF608A65D08A65E08A65D2208A6E3
:200C40005D08A65D08A65E08A65D2286F0E55EB5F002E55FF608A65E08A65D08A65D22080D
:200C6000A65F08A65E2286F0E55EB5F002E55FF608A65E08A65E2208A65D08A65E08A65E4A
:200C80002286F0E55EB5F002E55FF608A65D08A65D08A65D08A65D2208A65E08A65D08A685
:200CA0005E2286F0E55EB5F002E55FF608A65D08A65D08A65E2208A65D08A65D08A65D08AD
:200CC000A65E2290300D7820B146E520B4550AA3B146E520B4AA0280127554A57555F1B10F
:200CE000CDB109755400755500801D90300378807B0AB146A308DBFA90300F788C7B1AB16D
:200D000046A308DBFA90302922C2AFB189B1ABB1669030007400B14BA37411B14BA374CCAD
:200D2000B14B90300378807B0AB14AA308DBFA90300F788C7B1AB14AA308DBFAB19CB1BE5D
:200D4000B17A90302922E493F622E6438F01538FFDFFC3E58394F0400122EF8554B78555CC
:200D6000B7F0538FFE22438F02438F018554B78555B790300DF0538FFC2290300D7455B1FE
:200D80004B90300E74AAB14B227A3079D07820903040B146E520F709A3DAF7227A3079D0EE
:200DA000903040E7B14B09A3DAF9227A8C79007820903070B146E520F309A3DAF7227A8CD4
:200DC0007900903070E3B14B09A3DAF922788076FF0876330876010876010876190876FFBA
:200DE0000876090876600876010876FF08080876FF0876FF0876FF0876FF0876FF0876FF94
:200E00000876040876FF0876FF0876FF0876FF0876FF0876280876500876040876FF0876EE
:200E2000020876FF0876FF0876FF0876070876FF0876FF0876FF087600087600227888E639
:200E400014A2E19222A2E092217884745096500276507886740D965002760D863A789CE600
:200E60007539FFB402037539A0B4030375398275510078A0E6F8600674532409D8FCF551A4
:200E800078988653788DE6755000F54FB6FF03754FFF7883E624FF922978C076000876010E
:200EA00008761108762508765508765B08767708767F227554007555007597DE7597AD7595
:200EC00081B075EF0675A9001204827580FF75F1E175A4007580FF75D4FF75902A75F23F5C
:200EE00075A53F75902A75D5FF75A60175A72075F30175A70075E34075E202120482E4F8DF
:200F0000F6D8FDB1CD91C3D13DC2AF12037112044412046A120371C2AF75540075550012B9
:200F2000048275A91375A71075C10075A700780979007A0030850CDAFBD9F9D8F7120411AA
:200F400002F000302A0E12040A12037D12037D12037DC22A758851758E017589AA758C007A
:200F6000758D0075C80475910475D84075D90875F780759E0775960075DA4275DB42759BFD
:200F800080759D0075AF1875B90A75DF2F75BB1075E88575B22012035F31F375E4D5302742
:200FA0000375E45DC228C22475A82D75E68075B803D2AF758E0C755780755610755A507508
:200FC0005DF7755EE7755FD67563E17560EB7561CA7562A975300A120371E530602B75571F
:200FE000C0755608755A28755DFF755EF7755FEF7563E17560FB7561EB7562DA75300A124D
:201000000371E5306003020F17C0D075D010AF8ED0D0D22A753700C2AF1203B3D2AFC3E5F0
:2010200032940A40F9C2AF1203B9D2AFE4F541F542F55BF55CF533F53BC3E53B945E403355
:20104000753B000533789AE67814146012782814600D786414600878C8146003753300C303
:20106000E53398400E15337804C2AF12048212041DD2AF202806120AA01204D930250CE5B2
:20108000317003020F17120A0780AE1203712025A8C2AF120482D2AFE4F522F523F53812E4
:2010A000035F756500C2AF7984874E854E4C854E4D854E5275A71075C11075A70075A9039E
:2010C000C3E55733F557C3E55A33F55AC3E55633F556E55DC560F55DE55EC561F55EE55FD9
:2010E000C562F55F75633CD2AFA2219212302204A2269212D210D21175340075360C120977
:20110000B11209D212057512057C12057512057C1205751208051208E612092D12057C125B
:2011200007FA1204921208E612094E12057C1208051208E612096F12057C1207FA1208E6BB
:2011400012099012057C1208051208E61209B112057C1207FA1208E61209D212057C12042A
:20116000D930113530101A854E4CC3E5349418500530259F807EC210754CFF754DFF7552BE
:20118000FF201D15E53614600AF5363025852022828061C211D21C2113753700D21B3025D8
:2011A0001320220C79A4E76007C3E53294035044E5316040202209C3E54294F05036211335
:2011C000201D1220120520260580EC2026E9D21D854E4C213A854E4CC3E5429420400EC26D
:2011E0001DA2269212D211753612854E4C2113201B020537C2AFC2241204827522007523DC
:201200000075A91375A71075C10075A700D3E55713F557C3E55A13F55AC3E55613F556E50C
:201220005DC560F55DE55EC561F55EE55FC562F55F7563E1D2AF202517C3E53794045006FC
:20124000120371021091C2AF120416D2AF02100975370078A4E66006C291C293C295021007
:011260002C61
:202FE000FFFFFFFFFFFFFFFFFFFFFFFFFFFFFFFFFFFFFFFFFFFFFFFFFFFFFFFFFF020EB32B
:203000000011CCFFFF010132FF096001FF55AAFFFFFFFFFFFF04FFFFFFFFFF3B5004FF02B1
:20302000FFFFFF07FFFFFF0000FFFFFFFFFFFFFFFFFFFFFFFFFFFFFFFFFFFFFFFFFFFFFFA6
:2030400023415F585F303523202020202020202023424C48454C492445464D38423531239C
:20306000426C75656A6179202842455441292020023A042034420D00452D0D0034420D00D2
:203080004E27D300452DD01934190000000000000000000000000000000000000000000040
:2030A000000000000000000000000000000000000000000000000000000000000000000010
:2030C0000000000000000000000000000000000000000000000000000000000000000000F0
:2030E000000000000000000000000000000000000000FFFFFFFFFFFFFFFFFFFFFFFFFFFFDE
:10F00000C2AFC2D37597DE7597AD7581C075A90083
:10F0100075243875250331D87529A5752AF143F172
:10F020002053A4DFD28575D4FF75E3407DFA7803C1
:10F0300079E67C1075220075230090F1E57B06755A
:10F0400024987525013085020145208508D8FBD913
:10F05000F9DCF701B7308508D8FBD9F9DCF701B73F
:10F060003198E493A3C39A6004DDC301B7DBDB31BD
:10F070008A6002012E7B08E493FAA3316BDBF87AF5
:10F0800030316B752200752300318AEAFCEBFDC339
:10F09000ED94FE400E318A8A278B28ED30E0048AF9
:10F0A000828B83318A7AC270D8C3ED94FE60195086
:10F0B000CEBD0029EC600F7520007521FF75290079
:10F0C000752A000200000100A827A9280809D80411
:10F0D000D90201DA318EEAF201CE0D01A3C3ED941B
:10F0E000035051EDA2E092007AC5C3E5829400E599
:10F0F0008394F0508C200010438F02438F018529A8
:10F10000B7852AB7F0300027A827A9280809438F18
:10F1100001538FFDD804D902212FC3E58394F04019
:10F1200003A32114E28529B7852AB7F0A32114533C
:10F130008FFC017F7AC1BD030CE493A3FA314FDC4D
:10F14000F83147017F0181AA22AB23316BEBFAEA48
:10F150006222752608C3E52313F523E52213F52261
:10F1600050066323A0632201D526EA31D831D87531
:10F17000260AEAF4200102D285300102C28531D884
:10F18000C3134002C201D526EB22318EEAFB208553
:10F1900002218E3085022193752608AE24AF25C347
:10F1A000EF13FFEE13FE31DC31D8C3EA13308502D2
:10F1B0004480FA30E703632201C3E52313F523E516
:10F1C0002213F52250066323A0632201D526D9E538
:10F1D0002265236523F52222AE24AF250E0FDEFE25
:10F1E000DFFCD20122424C48656C6934373164E857
:03F1F000B5060160
:00000001FF
